:1000000064008510831685017F30810083126400AF
:1000100085018C0120308D003A308E006400060886
:1000200003108E0703188D0A8C0A0A300C02031D78
:100030000E28FF308C0064008B218B218B218B21BB
:100040008B218B218B218B218B218B218B218B2150
:100050008B218B21051285158B2105168B218B2178
:1000600005128B2105168B218B218B2105128B21EB
:1000700005168B218C1F05168C1B05128B21051272
:100080008B218B218B218B2105168B2105128B2136
:1000900005168B21051285118B2100000000000040
:1000A00085158B218B218B2105168B2105128B2128
:1000B0008D1D05128D1905168B210D1D05120D19AB
:1000C00005168B218D1C05128D1805168B210D1C14
:1000D00005120D1805168B218E1F05128E1B051695
:1000E0008B210E1F05120E1B05168B218E1E05126D
:1000F0008E1A05168B210E1E05120E1A05168B215F
:100100008E1D05128E1905168B210E1D05120E1956
